:1000000012C0189518951895189518951895189563
:1000100013C800C418951895189518951895189533
:100020001895189518958FE58DBFC8E3E0E24E2E20
:1000300084E08EBFD4E0F4E05F2EA89584B7082E4C
:10004000877F84BF88E1992781BD91BDEEEFF3E002
:10005000A0E6B0E088278D933197E9F76624A09851
:10006000A89AA198A99AA298AA9A8FEF81BB8FEF1C
:1000700087BBEAE1F0E0A4E9B0E091E0F0DE989916
:1000800057C081E08093620000916200083C10F04C
:1000900009F04EC000916200063909F03CC0809121
:1000A0008E00806880938E00A4E9B0E08C9198E087
:1000B00089278C93EAE1F0E0A4E9B0E091E07BE7E6
:1000C000BDDE00919400003009F00EC09298969821
:1000D000C798C2989098C6989798C598919A949AFC
:1000E000939AC19AC09A959A00919400083009F0A9
:1000F0000EC0929A969AC79AC29A909AC69A979A5E
:10010000C59A919894989398C198C09895988CEDB9
:1001100095E023DC0DC0989B01C00AC08AE090E006
:100120001CDCA2E6B0E08C918F5F8C9308F4ACCF1E
:10013000E4E1F0E0A0E1B0E08FDE0F3F09F05AC04B
:100140008EE591E0A7E7B0E08D939C938CE291E07F
:10015000A5E7B0E08D939C9388E191E0ADE7B0E036
:100160008D939C938AEF90E0ABE7B0E08D939C93E6
:1001700080E0809394008BEB809391008BEB8093D5
:100180009200E0E0F0E0A5E7B0E092E07BE756DE29
:10019000E5E0F0E0A7E7B0E092E07BE74FDEEAE0E1
:1001A000F0E0ABE7B0E092E07BE748DEEEE0F0E0C5
:1001B000ADE7B0E092E07BE741DEE0E1F0E0A1E90D
:1001C000B0E091E07BE73ADEE1E1F0E0A2E9B0E007
:1001D00091E07BE733DEEAE1F0E0A4E9B0E091E012
:1001E0007BE72CDEE4E1F0E0A0E1BB2784E68C9322
:1001F0007BE721DEE0E0F0E0A5E7B0E092E02FDE73
:10020000E5E0F0E0A7E7B0E092E029DEEAE0F0E028
:10021000ABE7B0E092E023DEEEE0F0E0ADE7B0E087
:1002200092E01DDEE0E1F0E0A1E9B0E091E017DE50
:10023000E1E1F0E0A2E9B0E091E011DE83E083BF0C
:1002400080E08FBD81E08EBD789489B7816089BFE1
:1002500089B7846089BF83E083BF81E08EBD85E07C
:1002600080939B0080918E00886080938E008091A7
:100270008E00846080938E0080E190E0A5E6B0E07F
:100280008D939C9385E090E0A7E6B0E08D939C93DE
:1002900081E090E0A9E6B0E08D939C9380E190E04E
:1002A000ABE6B0E08D939C9385E090E0ADE6B0E0E6
:1002B0008D939C9382E090E0AFE6B0E08D939C93A9
:1002C00081E08093B20084E08093B30083E0809368
:1002D000B40080ED97E041DB80918E00877F8093B2
:1002E0008E0080918E008B7F80938E00AFEAB0E00D
:1002F00082B78C93ADEAB0E08C9181FB81E00EF483
:1003000080E08F930091AF00023381E008F080E03D
:100310009F918923882309F421C0ABE9B0E08C9137
:10032000E3E31ADD81E08A93ABE9B0E08C916CECF9
:10033000BB27A6E1E3E332DD81E08A93ABE9B0E0DD
:100340008C9164E4BB27A6E1E3E328DD8091AD0056
:1003500082608093AD0080E08093AE00AFEAB0E0B1
:1003600082B78C93ADEAB0E08C9182FB81E00EF015
:1003700080E08F930091AF00023381E008F080E0CD
:100380009F918923882309F472C1ABE9B0E08C9175
:10039000E3E3E2DC81E08A93ABE9B0E08C916CECC2
:1003A000BB27A6E1E3E3FADC81E08A93ABE9B0E0A6
:1003B0008C916EEBBB27A6E1E3E3F0DCABE9B0E0A8
:1003C0008C91AEE9B0E0E3E329E02A9306DD88E012
:1003D000EEE9F0E04BDD402F0091A600041709F094
:1003E0001FC180919E0080939C0080919F0080930C
:1003F0009D0000919D00083F08F426C000E0409158
:100400009C00041BACE9B0E00C930FEF40919D0001
:10041000041BADE9B0E00C9362FA0EF414C0009135
:100420009B00053009F005C08091AD008064809389
:10043000AD0000919B00043009F005C08091AD0033
:1004400080628093AD0014C000919B00053009F0DC
:1004500005C08091AD008F7B8093AD0000919B0023
:10046000043009F005C08091AD008F7D8093AD0010
:10047000ECE8FEE125DCECE9F0E0D080EE24FF249E
:100480000027F0DA3BDBEDE0F0E0A7EAB0E0C7DC04
:10049000ADE9B0E00D91112740E150E06DDAABEA33
:1004A000B0E00D931C93EBEAF0E0D190E0808FEF89
:1004B000E7FE8827F82E082FD5DA05DBE7EAF0E01B
:1004C000ADDAACDBEDE0F0E0A7EAB0E0A8DCE0E913
:1004D000FEE1F6DBE7EAF0E0A1DA66DBEDE0F0E072
:1004E000A7EAB0E09CDC00919B00053009F005C054
:1004F000E7EAF0E0A5E9B0E092DC00919B0004306F
:1005000009F00AC0E7EAF0E04BDAA9E9B0E0EE0C46
:10051000000FE794DD92EC9262FA0EF453C0E5E925
:10052000F0E07CDAE4E9FEE1CBDBD3DB10F009F0AC
:1005300001C006C08091AD0080618093AD0005C010
:100540008091AD008F7E8093AD00A9E9B0E00D9160
:100550001C91073E53E0150714F009F001C006C0D6
:100560008091AD0088608093AD0005C08091AD00A2
:10057000877F8093AD00E5E9F0E012DAA1E7B0E013
:10058000EE0C000FE794DD92EC92A9E9B0E08D91BA
:100590009C91A9E7B0E08D939C9300919B0005305E
:1005A00009F005C080918E00816080938E000091DB
:1005B0009B00043009F005C08091AD0080688093F5
:1005C000AD002EC000919B00053081E009F080E075
:1005D0008F930091B000063981E008F080E09F9190
:1005E0008923882309F405C0A0EBB0E08C918F5FCC
:1005F0008C9300919B00043081E009F080E08F93A0
:100600000091B100063981E008F080E09F918923D4
:10061000882309F405C0A1EBB0E08C918F5F8C9327
:100620008091AD008B7F8093AD008091AD008D7F78
:100630008093AD0080E08093AE00AEE8B0E08C9196
:1006400081FB882780F9809580FBAEE8B0E08C9133
:1006500081F98C93AEE8B0E08C9181FB0EF004C080
:1006600084E080939B0003C085E080939B00ADEA0B
:10067000B0E08C9186FB0EF44DC0A7E7B0E04D9141
:100680005C91A5E7B0E00D911C910417150708F0E7
:1006900021C0A5E7B0E04D915C91A1E7B0E00D91DC
:1006A0001C910417150714F009F003C081E0809332
:1006B0007F00A7E7B0E04D915C91A1E7B0E00D911C
:1006C0001C91041715070CF001C003C080E0809353
:1006D0007F0020C0A5E7B0E04D915C91A1E7B0E0BC
:1006E0000D911C91041715070CF001C003C081E0A7
:1006F00080937F00A7E7B0E04D915C91A1E7B0E067
:100700000D911C910417150714F009F003C080E047
:1007100080937F0000917F00013081E009F080E04C
:100720008F93AEE8B0E08C9180FB81E00EF080E02A
:100730009F918923882309F402C0C39A01C0C398FA
:10074000ADEAB0E08C9185FB0EF44DC0ADE7B0E0B2
:100750004D915C91ABE7B0E00D911C91041715072A
:1007600008F021C0ABE7B0E04D915C91A9E7B0E0A3
:100770000D911C910417150714F009F003C081E0D6
:1007800080938000ADE7B0E04D915C91A9E7B0E0C7
:100790000D911C91041715070CF001C003C080E0F7
:1007A0008093800020C0ABE7B0E04D915C91A9E759
:1007B000B0E00D911C91041715070CF001C003C0A7
:1007C00081E080938000ADE7B0E04D915C91A9E7B6
:1007D000B0E00D911C910417150714F009F003C047
:1007E00080E08093800000918000013081E009F07A
:1007F00080E08F93ADEAB0E08C9187FB81E00EF052
:1008000080E09F918923882309F402C0C49A01C023
:10081000C4986CCD0F921F922F923F924F925F928D
:100820007F92AF92BF920F931F932F933F934F935B
:100830005F936F937F938F939F93AF93BF93CF9368
:10084000DF93EF93FF938FB78F93882783BF009138
:100850008D00003081E009F480E08F93AEE8B0E0D5
:100860008C9185FB81E00EF480E09F9189238823A1
:1008700009F403C0AFE8B0E01AD8AFE8B0E00D91DA
:100880001C9108355BE1150710F009F001C009C0A3
:1008900080E090E0AFE8B0E08D939C9380E080939F
:1008A0008D0000918D00003009F011C0A1E7B0E08B
:1008B0008D919C91A7E8B0E08D939C93A9E7B0E05F
:1008C0008D919C91A9E8B0E08D939C934FC001302D
:1008D00009F011C0A5E7B0E08D919C91A7E8B0E0C8
:1008E0008D939C93A9E7B0E08D919C91A9E8B0E02D
:1008F0008D939C933BC0023009F011C0A7E7B0E094
:100900008D919C91A7E8B0E08D939C93A9E7B0E00E
:100910008D919C91A9E8B0E08D939C9327C0033002
:1009200009F011C0A1E7B0E08D919C91A7E8B0E07B
:100930008D939C93ABE7B0E08D919C91A9E8B0E0DA
:100940008D939C9313C0043009F010C0A1E7B0E070
:100950008D919C91A7E8B0E08D939C93ADE7B0E0BA
:100960008D919C91A9E8B0E08D939C930091B0008B
:10097000043610F009F001C005C080918E00886037
:1009800080938E00AEE8B0E08C9183FB0EF4ABC098
:10099000A7E8B0E08D919C91A1E8B0E08D939C9385
:1009A000A1E8B0E08D919C91A5E8B0E08D939C9377
:1009B00083E0809363004091630001E0041710F02E
:1009C00009F025C0A1E8B0E00D911C914AE050E08B
:1009D00081D7A3E6B0E0AD90BB24A3E6B0E0AA0CBB
:1009E000BB1CAA0DBB1D0D931C93A1E8B0E00D919B
:1009F0001C914AE050E06ED7A1E8B0E04D935C93C3
:100A00008091630081508093630008F0D4CFA5E803
:100A1000B0E00D911C91043650E015070CF401C0B4
:100A200006C08BE090E0A5E6B0E08D939C93ADEA24
:100A3000B0E08C9186FB81E00EF080E08F93009116
:100A40008D00013081E009F480E09F9189238F932C
:100A500000918D00023081E009F480E09F918923AC
:100A6000882309F412C082E190E0A5E6B0E08D93FE
:100A70009C9381E190E0A7E6B0E08D939C938BE09E
:100A800090E0A9E6B0E08D939C93ADEAB0E08C9144
:100A900084FB81E00EF080E08F9300918D000130A7
:100AA00081E009F480E09F9189238F9300918D006C
:100AB000023081E009F480E09F918923882309F4C2
:100AC00012C083E190E0A5E6B0E08D939C9384E1B1
:100AD00090E0A7E6B0E08D939C938BE090E0A9E6D0
:100AE000B0E08D939C93AEE8B0E08C9182FB0EF465
:100AF000ABC0A9E8B0E08D919C91A3E8B0E08D93E4
:100B00009C93A3E8B0E08D919C91A5E8B0E08D9313
:100B10009C9386E0809363004091630004E0041797
:100B200010F009F025C0A3E8B0E00D911C914AE057
:100B300050E0D0D6A3E6B0E0AD90BB24A3E6B0E091
:100B4000AA0CBB1CAA0DBB1D0D931C93A3E8B0E01F
:100B50000D911C914AE050E0BDD6A3E8B0E04D9362
:100B60005C938091630081508093630008F0D4CF40
:100B7000A5E8B0E00D911C91043650E015070CF487
:100B800001C006C08BE090E0ABE6B0E08D939C9393
:100B9000ADEAB0E08C9185FB81E00EF080E08F93B0
:100BA00000918D00033081E009F480E09F9189235A
:100BB0008F9300918D00043081E009F480E09F91D3
:100BC0008923882309F412C082E190E0ABE6B0E00B
:100BD0008D939C9381E190E0ADE6B0E08D939C9382
:100BE0008BE090E0AFE6B0E08D939C93ADEAB0E08F
:100BF0008C9183FB81E00EF080E08F9300918D005B
:100C0000033081E009F480E09F9189238F93009164
:100C10008D00043081E009F480E09F9189238823CE
:100C200009F412C083E190E0ABE6B0E08D939C93B1
:100C300084E190E0ADE6B0E08D939C938BE090E092
:100C4000AFE6B0E08D939C9300919400003009F0E2
:100C500007C0919894989398C198C098959806C0A9
:100C6000919A949A939AC19AC09A959AA0E6B0E004
:100C70008C918F5F8C9300916000063010F009F02A
:100C800001C003C081E0809360009AD1A4E6B0E087
:100C90008C9186FBA2E3B0E08C9182F98C9390D189
:100CA000A4E6B0E08C9185FBA2E3B0E08C9186F9DC
:100CB0008C9386D1A4E6B0E08C9184FBA8E3B0E0ED
:100CC0008C9187F98C937CD1A4E6B0E08C9183FB66
:100CD000A8E3B0E08C9182F98C9372D1A4E6B0E0E5
:100CE0008C9182FBA2E3B0E08C9180F98C9368D167
:100CF000A4E6B0E08C9181FBA8E3B0E08C9186F98A
:100D00008C935ED1A4E6B0E08C9180FBA2E3B0E0CE
:100D10008C9187F98C9300916000013009F039C003
:100D200000919400003009F01DC0919AA3EBB0E04F
:100D30008C91A2E3B0E0FCD7F1D79C91982B9C93C7
:100D4000AEE8B0E08C9183FB0EF40AC0A1E9B0E0FC
:100D50008C9181FBA8E3B0E08C9185F98C9301C064
:100D6000C59A16C09198AEE8B0E08C9183FB0EF462
:100D70000EC0A1E9B0E08C9183FBA8E3B0E08C91B8
:100D800085F98C9388B390E2892788BB01C0C59808
:100D9000F9C0023009F02FC000919400003009F032
:100DA00013C0949AAEE8B0E08C9183FB0EF40AC0B5
:100DB000A1E9B0E08C9182FBA8E3B0E08C9185F9C9
:100DC0008C9301C0C59A16C09498AEE8B0E08C919F
:100DD00083FB0EF40EC0A1E9B0E08C9182FBA8E386
:100DE000B0E08C9185F98C9388B390E2892788BB19
:100DF00001C0C598C7C0033009F02FC0009194000E
:100E0000003009F013C0939AAEE8B0E08C9183FBF8
:100E10000EF40AC0A1E9B0E08C9183FBA8E3B0E036
:100E20008C9185F98C9301C0C59A16C09398AEE851
:100E3000B0E08C9183FB0EF40EC0A1E9B0E08C9180
:100E400081FBA8E3B0E08C9185F98C9388B390E2A4
:100E5000892788BB01C0C59895C0043009F02FC010
:100E600000919400003009F013C0C19AAEE8B0E0E0
:100E70008C9182FB0EF40AC0A2E9B0E08C9181FB58
:100E8000A8E3B0E08C9185F98C9301C0C59A16C097
:100E9000C198AEE8B0E08C9182FB0EF40EC0A2E9DE
:100EA000B0E08C9183FBA8E3B0E08C9185F98C9342
:100EB00088B390E2892788BB01C0C59863C005301C
:100EC00009F02FC000919400003009F013C0C09ABF
:100ED000AEE8B0E08C9182FB0EF40AC0A2E9B0E06B
:100EE0008C9182FBA8E3B0E08C9185F98C9301C0D2
:100EF000C59A16C0C098AEE8B0E08C9182FB0EF4A3
:100F00000EC0A2E9B0E08C9182FBA8E3B0E08C9126
:100F100085F98C9388B390E2892788BB01C0C59876
:100F200031C0063009F02EC000919400003009F065
:100F300013C0959AAEE8B0E08C9182FB0EF40AC023
:100F4000A2E9B0E08C9183FBA8E3B0E08C9185F935
:100F50008C9301C0C59A16C09598AEE8B0E08C910C
:100F600082FB0EF40EC0A2E9B0E08C9181FBA8E3F5
:100F7000B0E08C9185F98C9388B390E2892788BB87
:100F800001C0C59883E083BF8F918FBFFF91EF9120
:100F9000DF91CF91BF91AF919F918F917F916F9191
:100FA0005F914F913F912F911F910F91BF90AF9003
:100FB0007F905F904F903F902F901F900F901895CB
:100FC000A0E6B0E0AD90BB24A3E6B0E0AA0CBB1C49
:100FD000AA0DBB1D8C918093640000919400003099
:100FE00009F00AC0ECE0F0E1A4E6B0E08C919927AA
:100FF000A4E6B0E090D609C0E2E2F0E1A4E6B0E0F9
:101000008C919927A4E6B0E086D60895014F120688
:101010004C24200F00047E7F6A38307A42E2F1C807
:10102000FB007E306D79335B5F707F7B010015477D
:101030004F053D1D0E3704000F921F922F923F92D5
:101040004F925F927F92AF92BF920F931F932F9315
:101050003F934F935F936F937F938F939F93AF9340
:10106000BF93CF93DF93EF93FF938FB78F93A2E656
:10107000B0E08C918F5F8C93ADEAB0E08C9181FBF6
:1010800081E00EF080E08F930091AE000E3F81E092
:1010900008F080E09F918923882309F405C0AEEA17
:1010A000B0E08C918F5F8C930091AE00043110F012
:1010B00009F001C005C08091AD0084608093AD004F
:1010C0008EB5887F8EBDA3E3B0E00C9100FB81E07C
:1010D0000EF480E08F93AEE8B0E08C9187FB81E066
:1010E0000EF480E09F9189238F93A3E3B0E00C91ED
:1010F00001FB81E00EF080E09F9189238F93A3E3B1
:10110000B0E00C9102FB81E00EF080E09F9189231A
:10111000882309F401C0B4D0AEE8B0E08C9184FB20
:1011200081E00EF080E08F93A3E3B0E00C9100FB30
:1011300081E00EF080E09F918923882309F406C0A6
:10114000999901C0DED29A9901C02CD3A3E3B0E0F3
:101150000C9100FB81E00EF480E08F93A3E3B0E0FC
:101160000C9101FB81E00EF480E09F9189238F9325
:1011700000918D00003081E009F080E09F9189238B
:101180008F93AEE8B0E08C9186FB81E00EF480E0B6
:101190009F918923882309F401C05DD3A3E3B0E0C4
:1011A0000C9100FB81E00EF480E08F93A3E3B0E0AC
:1011B0000C9102FB81E00EF480E09F9189238F93D4
:1011C00000918D00003081E009F080E09F9189233B
:1011D0008F93AEE8B0E08C9186FB81E00EF480E066
:1011E0009F918923882309F401C04BD3A3E3B0E086
:1011F0000C9100FB81E00EF080E08F93A3E3B0E060
:101200000C9101FB81E00EF080E09F9189238F9388
:10121000A3E3B0E00C9102FB81E00EF080E09F912F
:101220008923882309F405C080918E008F778093ED
:101230008E00989B05C080918E008F7B80938E00DE
:1012400081E08EBD83E083BF8F918FBFFF91EF91CF
:10125000DF91CF91BF91AF919F918F917F916F91CE
:101260005F914F913F912F911F910F91BF90AF9040
:101270007F905F904F903F902F901F900F90189508
:10128000789489B7816089BF83E083BF80918E00A5
:10129000806180938E0080918E00806880938E00A4
:1012A00080E090E0AFE8B0E08D939C93A7E7B0E0DA
:1012B0004D915C91A5E7B0E00D911C9104171507C5
:1012C00081E009F080E08F93ADE7B0E04D915C9153
:1012D000ABE7B0E00D911C910417150781E009F010
:1012E00080E09F91892B882309F401C0FDD0ADE8EF
:1012F000B0E08C918F5F8C9300918D00043010F0E2
:1013000009F001C003C080E080938D0000918D0042
:10131000003009F043C080918E00886080938E0079
:1013200080918E00846080938E008AE090E0A5E634
:10133000B0E08D939C938AE090E0A7E6B0E08D93B7
:101340009C938AE090E0A9E6B0E08D939C938AE0BC
:1013500090E0ABE6B0E08D939C938AE090E0ADE640
:10136000B0E08D939C938AE090E0AFE6B0E08D937F
:101370009C9380918E008F7E80938E0084EF91E00D
:10138000ECD28EB5887F8EBD882783BFEEE0F0E07B
:10139000ADE7B0E092E07BE751D59BC0013009F0AA
:1013A0001BC080918E00886080938E0081E090E069
:1013B000A9E6B0E08D939C938CE090E0A7E6B0E0C6
:1013C0008D939C9380E090E0A5E6B0E08D939C9394
:1013D00084EF91E0C2D27DC0023009F027C0809135
:1013E0008E00886080938E0081E090E0A9E6B0E0F6
:1013F0008D939C938DE090E0A7E6B0E08D939C9355
:1014000080E090E0A5E6B0E08D939C9384EF91E0BE
:10141000A4D28EB5887F8EBD882783BFE0E0F0E040
:10142000A5E7B0E092E07BE709D553C0033009F0AF
:1014300027C080918E00846080938E0082E090E0CF
:10144000AFE6B0E08D939C938CE090E0ADE6B0E029
:101450008D939C9380E090E0ABE6B0E08D939C93FD
:1014600084EF91E07AD28EB5887F8EBD882783BFC6
:10147000E5E0F0E0A7E7B0E092E07BE7DFD429C049
:10148000043009F026C080918E00846080938E0025
:1014900082E090E0AFE6B0E08D939C938DE090E029
:1014A000ADE6B0E08D939C9380E090E0ABE6B0E0D9
:1014B0008D939C9384EF91E050D28EB5887F8EBD42
:1014C000882783BFEAE0F0E0ABE7B0E092E07BE79B
:1014D000B5D480918E00877F80938E0080918E009E
:1014E0008B7F80938E00089580918E008062809320
:1014F0008E00A7E7B0E04D915C91A5E7B0E00D91BB
:101500001C910417150709F059C080918E0088605E
:1015100080938E008FE090E0A5E6B0E08D939C93E1
:1015200080E190E0A7E6B0E08D939C9380E190E0AD
:10153000A9E6B0E08D939C9384EF91E00ED28BE00E
:1015400090E0A5E6B0E08D939C938BE090E0A7E659
:10155000B0E08D939C938BE090E0A9E6B0E08D9392
:101560009C9384EF91E0F9D18FE090E0A5E6B0E0A4
:101570008D939C9380E190E0A7E6B0E08D939C93DF
:1015800080E190E0A9E6B0E08D939C9384EF91E038
:10159000E4D18BE090E0A5E6B0E08D939C938BE0E6
:1015A00090E0A7E6B0E08D939C938BE090E0A9E6F5
:1015B000B0E08D939C9384EF91E0CFD1ADE7B0E0A4
:1015C0004D915C91ABE7B0E00D911C9104171507AC
:1015D00009F059C080918E00846080938E008FE066
:1015E00090E0ABE6B0E08D939C9380E190E0ADE6B7
:1015F000B0E08D939C9380E190E0AFE6B0E08D93F6
:101600009C9384EF91E0A9D18BE090E0ABE6B0E051
:101610008D939C938BE090E0ADE6B0E08D939C932E
:101620008BE090E0AFE6B0E08D939C9384EF91E087
:1016300094D18FE090E0ABE6B0E08D939C9380E195
:1016400090E0ADE6B0E08D939C9380E190E0AFE652
:10165000B0E08D939C9384EF91E07FD18BE090E09C
:10166000ABE6B0E08D939C938BE090E0ADE6B0E00C
:101670008D939C938BE090E0AFE6B0E08D939C93CC
:1016800084EF91E06AD100918D00003009F001C033
:1016900027C0013009F007C0E0E0F0E0A5E7B0E0C6
:1016A00092E0DDD31DC0023009F007C0E5E0F0E0B4
:1016B000A7E7B0E092E0D3D313C0033009F007C02E
:1016C000EAE0F0E0ABE7B0E092E0C9D309C0043053
:1016D00009F006C0EEE0F0E0ADE7B0E092E0BFD385
:1016E00080918D00815080938D0080E090E0AFE884
:1016F000B0E08D939C9380918E008F7D80938E00BF
:101700000895789489B7816089BF83E083BF80E0C2
:1017100090E0AFE8B0E08D939C9300918D00013094
:1017200009F00DC0A5E7B0E00D911C91073E53E014
:10173000150708F003C0A5E7B0E0B9D02FC002300C
:1017400009F00DC0A7E7B0E00D911C91073E53E0F2
:10175000150708F003C0A7E7B0E0A9D01FC0033009
:1017600009F00DC0ABE7B0E00D911C91073E53E0CE
:10177000150708F003C0ABE7B0E099D00FC0043004
:1017800009F00CC0ADE7B0E00D911C91073E53E0AD
:10179000150708F003C0ADE7B0E089D08EE190E016
:1017A000DCD00895789489B7816089BF83E083BFD6
:1017B00080E090E0AFE8B0E08D939C9300918D00C5
:1017C000013009F00FC0A5E7B0E00D911C91003089
:1017D00050E0150710F009F001C003C0A5E7B0E024
:1017E0006DD035C0023009F00FC0A7E7B0E00D9111
:1017F0001C91003050E0150710F009F001C003C043
:10180000A7E7B0E05BD023C0033009F00FC0ABE71F
:10181000B0E00D911C91003050E0150710F009F078
:1018200001C003C0ABE7B0E049D011C0043009F0FB
:101830000EC0ADE7B0E00D911C91003050E01507EF
:1018400010F009F001C003C0ADE7B0E037D08EE181
:1018500090E083D0089580918E00806480938E0004
:1018600091E0A1E9B0E092D08EB5887F8EBD882747
:1018700083BFE0E1F0E0A1E9B0E091E07BE7DED2F8
:10188000089580918E00806480938E0091E0A2E99B
:10189000B0E07CD08EB5887F8EBD882783BFE1E124
:1018A000F0E0A2E9B0E091E07BE7C8D20895ED91C5
:1018B000FC91EF5FFF4FFC93EE930895ED91FC9147
:1018C000E150F040FC93EE93089508D055D000FC11
:1018D00010D0089503D01ED001F8F9CF0024E89469
:1018E00057FF02C009D0689400F80BD010F801240B
:1018F000089502D009D00895509540954F5F5F4FED
:101900000895E89417FF0895009510950F5F1F4FF5
:1019100068940895352F242FE894452B11F468948A
:101920000895512F402F0027112780E1440F551FA4
:10193000001F111F021B130B416018F4020F131F2D
:101940004E7F8A9599F708953197F1F70895689435
:1019500062F80895E89462F80895EF93FF93EE27F4
:10196000E82BE92B31F0E0EDF7E03197F1F7019743
:10197000D1F7FF91EF9108950F92B801469F800132
:10198000479F100D569F100D0F900895903039F01D
:101990008C91880F08F481609A95D9F78C930895FB
:1019A0003DD0992711278F2D880F80E8F82A802FA6
:1019B000881F08F41FEF41F08F57082F07FD04C060
:1019C000003240F08FEF01C08827982FD82EE82EE4
:1019D000F82E09C08FE1801B082FF694E794D79466
:1019E00097950A95D1F7112351F09095D094E094F2
:1019F000F09481E0980F8827D81EE81EF81E0F2D5E
:101A0000FE2CED2CD92E0895D094E094F09491E022
:101A1000D90E9927E91EF91E10950895D190E190ED
:101A2000F190019108952191319141915191089541
:101A3000102F90E8FF0C001F0927990FF7941078DA
:101A4000652F90E8440F551F5927990F47956078E7
:101A500000380895FF0C90E89027110F9795F794A0
:101A6000092F0895102FBD2CDE2CEF2CF02E112302
:101A70004AF4B094D094E094F0949FEFB91AD90A44
:101A8000E90AF90A0EE1FF2039F4FE2CED2CDB2CDB
:101A9000BB240850C2F766C032F00A95BB0CDD1CAF
:101AA000EE1CFF1CF9CF01D0D5CFB7FE089590E80A
:101AB000B91611F4D0FE08959FEFD91AE90AF90A70
:101AC00009F403950895502F2D2D3E2D4F2D612F94
:101AD00008952DEC3CEC4CEC5DE366270FC09EDFD7
:101AE000F2DFDD24EE2490E8F92E0FE307C09BDF40
:101AF00005C02227332740E251E46627552351F1E0
:101B0000002381F195DF71F1162700585058089491
:101B1000050B18F407FD03C025C007FD23C046953B
:101B200037952795F694E794D79422D0FF202AF092
:101B3000DD0CEE1CFF1C015073F09D2D969548F0B6
:101B4000DD203AF4EE202AF491E0D90E9927E91E1F
:101B5000F91E80CF07C09FE7092FF92A9FEFD92EE2
:101B6000E92E0895DD24EE24FF240027112708958F
:101B70009F929924AA24BB2488E1D216E306F40696
:101B800028F0D21AE30AF40A089401C08894991C38
:101B9000AA1CBB1CDD0CEE1CFF1C8A9571F7D92C0E
:101BA000EA2CFB2C9F90089543DFE1F25038D1F2EC
:101BB0001627005850580894051F12F418F4CBCF7C
:101BC00008F0D0CF0BD0FF202AF0BB0CDD1CEE1CA0
:101BD000FF1C40CF0F5F0BF4BECF3CCF9F929924E8
:101BE000AA24BB24992788E1990CAA1CBB1CDD1CE4
:101BF000EE1CFF1C30F4920EA31EB41ED91EE91E6B
:101C0000F91E8A9589F79F9008950AF045D022CF52
:101C10005FE322273327442701C005DF09DF50385F
:101C2000B1F3003899F3902F951B8BF312F434D055
:101C3000FACF983118F0222733274427983028F01C
:101C4000232F342F44279850F9CF992329F0469514
:101C5000379527959A95D9F7912F962742F014D06A
:101C6000B0F6F794E794D7940F5F8BF674CF10D04B
:101C700051F008F4C9DEFF2052F2DD0CEE1CFF1C0F
:101C80000150CBF768CF6ECFD20EE31EF41E08953D
:101C9000D21AE30AF40A0895DF92EF92FF920F93AB
:101CA0001F93D22EE32EF42E052F162F6F915F91E6
:101CB0004F913F912F910895C89531960020089536
:101CC000FBDF202DF9DF302DF7DF402DF5DF502D24
:101CD000089507FB00680EF40F7757FB50680EF469
:101CE0005F7707FD02C057FF05C0D216E306F40672
:101CF000050708952D153E054F055007089591E0FD
:101D000005C092E003C094E001C098E0D5DF0D92D9
:101D10009A95E1F70895E80FF91FF1CF91E0882334
:101D200021F08894991F8A95E9F7892F9095089555
:101D3000883018F011968850FBCF08950181082B48
:101D40000183128119231283EF93FF93E8E0F0E0FF
:101D5000FBDDFF91EF910895FDDDFF27DFDFEEDF73
:101D6000EF93FF93ECEBF3E0EFDDFF91EF91182B96
:101D7000128309230183EF93FF93E8E8F0E0E4DDA9
:101D8000FF91EF911081182309F0E1DDEF93FF93AC
:101D9000E0E3F3E0D9DDFF91EF910895BFDFFF2786
:101DA00029915D9148E0CADF579510F4182B1283F2
:101DB000EF93FF93E8E6F0E0C7DDFF91EF91182B7A
:101DC0001283EF93FF93E0E1F0E0BEDDFF91EF912E
:101DD0004A9549F72A9529F70895A0DFFF27299109
:101DE00048E05527ABDF09230183EF93FF93EEE033
:101DF000F0E0AADDFF91EF9188941081182309F09B
:101E000008945795EF93FF93EAE6F0E09DDDFF918C
:101E1000EF914A9539F75D932A9511F7089594E06B
:101E200081918D939A95E1F70895E199FECFEEBBEC
:101E3000FFBB3196089591E001C092E07B3751F4E9
:101E40007FB7F894F2DF8D918DBBE29AE19A9A9573
:101E5000C9F77FBF7727089591E001C092E0E5DFE1
:101E6000E09A8DB38D939A95D1F7089500276CE889
:101E7000719198E00695779577FF18F477FD08F053
:101E800006279A95B9F78A9599F708950000804139
:081E90000000204100C079446C
:00000001FF
